:0200000480007A
:100000006F000005732F2034930F80006308FF03F7
:10001000930F90006304FF03930FB0006300FF038E
:10002000130F000063040F0067000F00732F2034CC
:1000300063540F006F00400093E19153171F0000BD
:1000400023223FFC171F000023200FFC6FF01FFF2F
:100050009300000013010000930100001302000050
:100060009302000013030000930300001304000038
:100070009304000013050000930500001306000020
:100080009306000013070000930700001308000008
:10009000930800001309000093090000130A0000F0
:1000A000930A0000130B0000930B0000130C0000D8
:1000B000930C0000130D0000930D0000130E0000C0
:1000C000930E0000130F0000930F0000732540F102
:1000D0006310050097020000938202017390523072
:1000E000735044749702000093820201739052305F
:1000F00073500018970200009382020273905230EE
:10010000B70200809382F2FF7390023B9302F001EA
:100110007390023A7350403097020000938242017C
:100120007390523073502030735030309301000080
:1001300097020000938242ED739052301305100035
:100140001315F501634C05000F00F00F930110002B
:100150009308D0051305000073000000930200000F
:10016000638A020073905210B7B20000938292101B
:100170007390223073500030970200009382420146
:1001800073901234732540F17300203093012000E6
:10019000930000001301100063962000631A302AB8
:1001A00063163000E39E20FE6314302A9301300072
:1001B000930010001301000063962000631A30289A
:1001C00063163000E39E20FE631430289301400044
:1001D0009300F0FF1301100063962000631A30268D
:1001E00063163000E39E20FE631430269301500016
:1001F000930010001301F0FF63962000631A30246F
:1002000063163000E39E20FE6314302493016000E7
:100210009300000013010000639420006314300079
:1002200063183022E39E20FE9301700093001000BB
:10023000130110006394200063143000631A30200F
:10024000E39E20FE930180009300F0FF1301F0FF76
:100250006394200063143000631C301EE39E20FE74
:1002600093019000130200009300000013010000AE
:100270006390201E1302120093022000E31652FE28
:100280009301A0001302000093000000130100007E
:1002900013000000639E201A130212009302200034
:1002A000E31452FE9301B00013020000930000001B
:1002B000130100001300000013000000639A2018CF
:1002C0001302120093022000E31252FE9301C000B9
:1002D000130200009300000013000000130100004F
:1002E000639820161302120093022000E31452FEBA
:1002F0009301D000130200009300000013000000DF
:100300001301000013000000639420141302120074
:1003100093022000E31252FE9301E000130200005A
:100320009300000013000000130000001301000000
:10033000639020121302120093022000E31252FE77
:100340009301F0001302000093000000130100006D
:10035000639020101302120093022000E31652FE55
:10036000930100011302000093000000130100003C
:1003700013000000639E200C130212009302200061
:10038000E31452FE930110011302000093000000D9
:10039000130100001300000013000000639A200AFC
:1003A0001302120093022000E31252FE9301200177
:1003B000130200009300000013000000130100006E
:1003C000639820081302120093022000E31452FEE7
:1003D000930130011302000093000000130000009D
:1003E00013010000130000006394200613021200A2
:1003F00093022000E31252FE930140011302000019
:10040000930000001300000013000000130100001F
:10041000639020041302120093022000E31252FEA4
:100420009301500193001000639A00009380100024
:100430009380100093801000938010009380100030
:1004400093801000930330006394700063103002B7
:100450000F00F00F638001009391110093E11100F0
:100460009308D00513850100730000000F00F00F02
:10047000930110009308D0051305000073000000DD
:10048000731000C000000000000000000000000029
:10049000000000000000000000000000000000005C
:1004A000000000000000000000000000000000004C
:0C04B00000000000000000000000000040
:1010000000000000000000000000000000000000E0
:1010100000000000000000000000000000000000D0
:1010200000000000000000000000000000000000C0
:1010300000000000000000000000000000000000B0
:081040000000000000000000A8
:040000058000000077
:00000001FF
